
 TEST

 Start     Length     Name                   Class
 0001:0000 040C0H     _TEXT                  CODE
 0002:0000 00010H     NULL                   BEGDATA
 0002:0010 00B1CH     _DATA                  DATA
 0002:0B2C 0000EH     CDATA                  DATA
 0002:0B3A 00000H     XIFB                   DATA
 0002:0B3A 00000H     XIF                    DATA
 0002:0B3A 00000H     XIFE                   DATA
 0002:0B3A 00000H     XIB                    DATA
 0002:0B3A 00000H     XI                     DATA
 0002:0B3A 00000H     XIE                    DATA
 0002:0B3A 00000H     XPB                    DATA
 0002:0B3A 00002H     XP                     DATA
 0002:0B3C 00000H     XPE                    DATA
 0002:0B3C 00000H     XCB                    DATA
 0002:0B3C 00000H     XC                     DATA
 0002:0B3C 00000H     XCE                    DATA
 0002:0B3C 00000H     XCFB                   DATA
 0002:0B3C 00000H     XCF                    DATA
 0002:0B3C 00000H     XCFE                   DATA
 0002:0B3C 0000CH     DBDATA                 DATA
 0002:0B48 00002H     XIQC                   DATA
 0002:0B4A 00000H     CONST                  CONST
 0002:0B4A 00019H     HDR                    MSG
 0002:0B63 000B1H     MSG                    MSG
 0002:0C14 00002H     PAD                    MSG
 0002:0C16 00001H     EPAD                   MSG
 0002:0C20 00020H     _BSS                   BSS
 0002:0C40 00000H     XOB                    BSS
 0002:0C40 00000H     XO                     BSS
 0002:0C40 00000H     XOE                    BSS
 0002:0C40 001B4H     c_common               BSS

 Origin   Group
 0002:0   DGROUP

 Address   Export                  Alias

 0001:24CB FAULTDIALOGPROC         FAULTDIALOGPROC
 0001:0868 MEMWNDPROC              MEMWNDPROC
 0001:2670 MYFAULTHANDLER          MYFAULTHANDLER
 0001:238C MYNOTIFYHANDLER         MYNOTIFYHANDLER
 0001:0226 WndProc                 WndProc

  Address         Publics by Name

 0000:0000  Imp  APPENDMENU           (USER.411)
 0000:0000  Imp  BEGINPAINT           (USER.39)
 0000:0000  Imp  CHECKMENUITEM        (USER.154)
 0000:0000  Imp  CLASSFIRST           (TOOLHELP.20)
 0000:0000  Imp  CLASSNEXT            (TOOLHELP.21)
 0000:0000  Imp  CREATEWINDOW         (USER.41)
 0000:0000  Imp  DEFWINDOWPROC        (USER.107)
 0000:0000  Imp  DELETEOBJECT         (GDI.69)
 0000:0000  Imp  DIALOGBOX            (USER.87)
 0000:0000  Imp  DISPATCHMESSAGE      (USER.114)
 0001:0EC4       DUMPMEM
 0000:0000  Imp  ENDDIALOG            (USER.88)
 0000:0000  Imp  ENDPAINT             (USER.40)
 0000:0000  Imp  FATALAPPEXIT         (KERNEL.137)
 0000:0000  Imp  FATALEXIT            (KERNEL.1)
 0001:25F4       FAULT
 0001:24CB       FAULTDIALOGPROC
 0000:0000  Imp  FREEPROCINSTANCE     (KERNEL.52)
 0000:0000  Imp  GDIHEAPINFO          (TOOLHELP.23)
 0000:0000  Imp  GETCLIENTRECT        (USER.33)
 0000:0000  Imp  GETCURRENTTASK       (KERNEL.36)
 0000:0000  Imp  GETDC                (USER.66)
 0000:0000  Imp  GETMENU              (USER.157)
 0000:0000  Imp  GETMENUSTATE         (USER.250)
 0000:0000  Imp  GETMESSAGE           (USER.108)
 0000:0000  Imp  GETMODULEHANDLE      (KERNEL.47)
 0000:0000  Imp  GETSCROLLPOS         (USER.63)
 0000:0000  Imp  GETSCROLLRANGE       (USER.65)
 0000:0000  Imp  GETSTOCKOBJECT       (GDI.87)
 0000:0000  Imp  GETSYSTEMMENU        (USER.156)
 0000:0000  Imp  GETSYSTEMMETRICS     (USER.179)
 0000:0000  Imp  GETTEXTMETRICS       (GDI.93)
 0000:0000  Imp  GETWINDOWLONG        (USER.135)
 0000:0000  Imp  GETWINDOWWORD        (USER.133)
 0000:0000  Imp  GLOBALALLOC          (KERNEL.15)
 0000:0000  Imp  GLOBALENTRYHANDLE    (TOOLHELP.5)
 0000:0000  Imp  GLOBALENTRYMODULE    (TOOLHELP.6)
 0000:0000  Imp  GLOBALFIRST          (TOOLHELP.2)
 0000:0000  Imp  GLOBALFREE           (KERNEL.17)
 0000:0000  Imp  GLOBALINFO           (TOOLHELP.4)
 0000:0000  Imp  GLOBALLOCK           (KERNEL.18)
 0000:0000  Imp  GLOBALNEXT           (TOOLHELP.3)
 0000:0000  Imp  GLOBALREALLOC        (KERNEL.16)
 0000:0000  Imp  GLOBALUNLOCK         (KERNEL.19)
 0000:0000  Imp  INITAPP              (USER.5)
 0000:0000  Imp  INITTASK             (KERNEL.91)
 0000:0000  Imp  INTERRUPTREGISTER    (TOOLHELP.27)
 0000:0000  Imp  INTERRUPTUNREGISTER  (TOOLHELP.28)
 0000:0000  Imp  INVALIDATERECT       (USER.125)
 0000:0000  Imp  LOADCURSOR           (USER.173)
 0000:0000  Imp  LOADICON             (USER.174)
 0000:0000  Imp  LOCALALLOC           (KERNEL.5)
 0000:0000  Imp  LOCALFIRST           (TOOLHELP.8)
 0000:0000  Imp  LOCALFREE            (KERNEL.7)
 0000:0000  Imp  LOCALINFO            (TOOLHELP.7)
 0000:0000  Imp  LOCALNEXT            (TOOLHELP.9)
 0000:0000  Imp  LOCALREALLOC         (KERNEL.6)
 0000:0000  Imp  LOCKSEGMENT          (KERNEL.23)
 0000:0000  Imp  LSTRCPY              (KERNEL.88)
 0000:0000  Imp  MAKEPROCINSTANCE     (KERNEL.51)
 0000:0000  Imp  MEMMANINFO           (TOOLHELP.24)
 0000:0000  Imp  MEMORYREAD           (TOOLHELP.30)
 0000:0000  Imp  MEMORYWRITE          (TOOLHELP.31)
 0001:0868       MEMWNDPROC
 0000:0000  Imp  MESSAGEBOX           (USER.1)
 0000:0000  Imp  MODULEFINDHANDLE     (TOOLHELP.13)
 0000:0000  Imp  MODULEFIRST          (TOOLHELP.10)
 0000:0000  Imp  MODULENEXT           (TOOLHELP.11)
 0000:0000  Imp  MOVEWINDOW           (USER.56)
 0001:2670       MYFAULTHANDLER
 0001:238C       MYNOTIFYHANDLER
 0000:0000  Imp  NOTIFYREGISTER       (TOOLHELP.25)
 0000:0000  Imp  NOTIFYUNREGISTER     (TOOLHELP.26)
 0000:0000  Imp  OUTPUTDEBUGSTRING    (KERNEL.115)
 0000:0008  Abs  pAtomTable
 0000:0006  Abs  PLOCALHEAP
 0000:0000  Imp  POSTMESSAGE          (USER.110)
 0000:0000  Imp  POSTQUITMESSAGE      (USER.6)
 0000:000E  Abs  pStackBot
 0000:000C  Abs  pStackMin
 0000:000A  Abs  pStackTop
 0000:0000  Imp  REGISTERCLASS        (USER.57)
 0000:0000  Imp  RELEASEDC            (USER.68)
 0002:0004       rsrvptrs
 0000:0000  Imp  SCROLLWINDOW         (USER.61)
 0000:0000  Imp  SELECTOBJECT         (GDI.45)
 0000:0000  Imp  SENDMESSAGE          (USER.111)
 0000:0000  Imp  SETCURSOR            (USER.69)
 0000:0000  Imp  SETDLGITEMTEXT       (USER.92)
 0000:0000  Imp  SETSCROLLPOS         (USER.62)
 0000:0000  Imp  SETSCROLLRANGE       (USER.64)
 0000:0000  Imp  SETWINDOWLONG        (USER.136)
 0000:0000  Imp  SETWINDOWTEXT        (USER.37)
 0000:0000  Imp  SETWINDOWWORD        (USER.134)
 0000:0000  Imp  SHOWCURSOR           (USER.71)
 0000:0000  Imp  SHOWWINDOW           (USER.42)
 0000:0000  Imp  STACKTRACEFIRST      (TOOLHELP.17)
 0000:0000  Imp  STACKTRACENEXT       (TOOLHELP.19)
 0002:0930       STKHQQ
 0000:0000  Imp  TASKFINDHANDLE       (TOOLHELP.16)
 0000:0000  Imp  TASKFIRST            (TOOLHELP.14)
 0000:0000  Imp  TASKNEXT             (TOOLHELP.15)
 0000:0000  Imp  TERMINATEAPP         (TOOLHELP.29)
 0000:0000  Imp  TEXTOUT              (GDI.33)
 0000:0000  Imp  TIMERCOUNT           (TOOLHELP.32)
 0000:0000  Imp  TRANSLATEMESSAGE     (USER.113)
 0000:0000  Imp  UNLOCKSEGMENT        (KERNEL.24)
 0000:0000  Imp  UPDATEWINDOW         (USER.124)
 0000:0000  Imp  USERHEAPINFO         (TOOLHELP.22)
 0000:0000  Imp  WAITEVENT            (KERNEL.30)
 0001:0010       WINMAIN
 0001:0226       WndProc
 0002:0260       _bHasData
 0001:1EA5       _DoGDIInfo
 0001:21E8       _DoGlobalEntryModuleTest
 0001:1FCA       _DoMemManInfo
 0001:1C1B       _DoStackTrace
 0001:1D80       _DoUserInfo
 0002:0C20       _edata
 0002:0DF4       _end
 0002:097F       _environ
 0002:0958       _errno
 0001:2899       _exit
 0001:3FF6       _fflush
 0001:4068       _flushall
 0002:0C40       _hInst
 0002:0DE6       _hwndList
 0002:0DE8       _hwndListLocal
 0002:0D38       _hwndListStatic
 0002:0DDC       _hwndMain
 0001:3B20       _lseek
 0001:3EA0       _malloc
 0001:3CD8       _memset
 0001:2411       _MyCFaultHandler
 0001:3D9C       _read
 0001:225E       _ReadMemoryTest
 0001:275C       _sprintf
 0001:27B2       _sscanf
 0001:3E8E       _stackavail
 0001:270E       _strcpy
 0001:2740       _strlen
 0002:0236       _szAppName
 0002:024A       _szBlockTypes
 0002:0276       _szGDI
 0002:026C       _szLocalFlags
 0002:023E       _szMemName
 0002:02C2       _szNotify
 0002:0CE8       _szText
 0002:028E       _szUser
 0001:230F       _TimerCountTest
 0001:3AC0       _ungetc
 0001:1B1A       _WalkClassList
 0001:1328       _WalkFreeList
 0001:10B0       _WalkGlobalHeap
 0001:1738       _WalkLocalHeap
 0001:1530       _WalkLRUList
 0001:1914       _WalkModuleList
 0001:1A16       _WalkTaskList
 0002:0DE0       _wFilterState
 0002:0234       _wListStatus
 0002:0DDA       _wNotifyIn
 0002:0CE6       _wNotifyOut
 0002:0DF2       _wNotifyState
 0001:3B9A       _write
 0002:0DE4       _wsCS
 0002:0CE4       _wsFault
 0002:0DDE       _wsFaultTask
 0002:0DE2       _wsIP
 0000:0000  Imp  _wsprintf            (USER.420)
 0002:0CE2       _wsProgramTask
 0002:0DEA       _xChar
 0002:0DEC       _xScreen
 0002:0DEE       _yChar
 0002:0DF0       _yScreen
 0002:09FC       __aaltstkovr
 0002:093C       __acfinfo
 0000:9876  Abs  __acrtmsg
 0000:9876  Abs  __acrtused
 0000:9876  Abs  __acrtused2
 0000:D6D6  Abs  __aDBdoswp
 0002:098E       __adbgmsg
 0002:0B40       __aDBrterr
 0001:3916       __aFchkstk
 0000:0000  Imp  __AHINCR             (KERNEL.114)
 0002:094A       __aintdiv
 0002:0B28       __amblksiz
 0001:394F       __amsg_exit
 0001:38F6       __aNchkstk
 0001:3D06       __aNFalmul
 0001:3D28       __aNFalshl
 0001:3D06       __aNFaulmul
 0001:3FB8       __aNlmul
 0001:3FEA       __aNlshl
 0001:3FB8       __aNulmul
 0002:0A0E       __asizeC
 0002:0A0F       __asizeD
 0001:26A1       __astart
 0002:0B52       __caption
 0001:28A8       __cexit
 0002:09FE       __cfltcvt_tab
 0002:0B26       __cflush
 0002:0986       __child
 0001:38F6       __chkstk
 0001:27EC       __cinit
 0001:394A       __cintDIV
 0001:2902       __ctermsub
 0002:0A10       __ctype
 0002:0A10       __ctype_
 0001:28B2       __c_exit
 0002:0963       __doserrno
 0001:3D46       __dosret0
 0001:3D5B       __dosretax
 0001:3D4E       __dosreturn
 0002:0960       __dosvermajor
 0002:0961       __dosverminor
 0001:28A0       __exit
 0002:094E       __fac
 0001:3F18       __ffree
 0001:39EA       __filbuf
 0001:2B5E       __flsbuf
 0001:3EEE       __fmalloc
 0002:0B2E       __fpinit
 0000:9876  Abs  __fptaskdata
 0001:38F0       __fptrap
 0001:3F78       __frealloc
 0001:3A7E       __getbuf
 0001:2C3E       __input
 0002:0989       __intno
 0002:0D3A       __iob
 0002:0C42       __iob2
 0002:0B2A       __lastiob
 0001:3D68       __maperror
 0001:39BE       __myalloc
 0002:0965       __nfile
 0001:3EDE       __nfree
 0001:3EA4       __nmalloc
 0001:396C       __NMSG_TEXT
 0001:3997       __NMSG_WRITE
 0001:3F28       __nrealloc
 0002:0963       __oserr
 0002:0967       __osfile
 0002:0960       __osmajor
 0002:0961       __osminor
 0002:0962       __osmode
 0002:0960       __osversion
 0001:341A       __output
 0002:0988       __ovlflag
 0002:098A       __ovlvec
 0002:0981       __pgmptr
 0002:095E       __psp
 0002:095C       __pspadr
 0001:2952       __setargv
 0001:2AE0       __setenvp
 0002:0A0C       __sigintoff
 0002:0A0A       __sigintseg
 0002:095A       __umaskval
 0002:0B42       ___aDBexit
 0002:0B3E       ___aDBswpchk
 0002:0B3C       ___aDBswpflg
 0002:097B       ___argc
 0002:097D       ___argv
 0002:0B48       ___qczrinit

  Address         Publics by Value

 0000:0000  Imp  TIMERCOUNT           (TOOLHELP.32)
 0000:0000  Imp  SETDLGITEMTEXT       (USER.92)
 0000:0000  Imp  GLOBALFIRST          (TOOLHELP.2)
 0000:0000  Imp  ENDDIALOG            (USER.88)
 0000:0000  Imp  GLOBALUNLOCK         (KERNEL.19)
 0000:0000  Imp  MEMMANINFO           (TOOLHELP.24)
 0000:0000  Imp  DEFWINDOWPROC        (USER.107)
 0000:0000  Imp  SETWINDOWTEXT        (USER.37)
 0000:0000  Imp  DISPATCHMESSAGE      (USER.114)
 0000:0000  Imp  SETWINDOWLONG        (USER.136)
 0000:0000  Imp  TEXTOUT              (GDI.33)
 0000:0000  Imp  STACKTRACEFIRST      (TOOLHELP.17)
 0000:0000  Imp  SHOWWINDOW           (USER.42)
 0000:0000  Imp  LSTRCPY              (KERNEL.88)
 0000:0000  Imp  MEMORYWRITE          (TOOLHELP.31)
 0000:0000  Imp  GETTEXTMETRICS       (GDI.93)
 0000:0000  Imp  GETMESSAGE           (USER.108)
 0000:0000  Imp  GETCURRENTTASK       (KERNEL.36)
 0000:0000  Imp  FATALAPPEXIT         (KERNEL.137)
 0000:0000  Imp  LOCALFIRST           (TOOLHELP.8)
 0000:0000  Imp  GLOBALINFO           (TOOLHELP.4)
 0000:0000  Imp  GLOBALLOCK           (KERNEL.18)
 0000:0000  Imp  GETSCROLLPOS         (USER.63)
 0000:0000  Imp  POSTMESSAGE          (USER.110)
 0000:0000  Imp  MEMORYREAD           (TOOLHELP.30)
 0000:0000  Imp  SETSCROLLPOS         (USER.62)
 0000:0000  Imp  CREATEWINDOW         (USER.41)
 0000:0000  Imp  GETWINDOWWORD        (USER.133)
 0000:0000  Imp  TASKNEXT             (TOOLHELP.15)
 0000:0000  Imp  GLOBALALLOC          (KERNEL.15)
 0000:0000  Imp  GETMENU              (USER.157)
 0000:0000  Imp  MODULEFIRST          (TOOLHELP.10)
 0000:0000  Imp  GETWINDOWLONG        (USER.135)
 0000:0000  Imp  GETSCROLLRANGE       (USER.65)
 0000:0000  Imp  UNLOCKSEGMENT        (KERNEL.24)
 0000:0000  Imp  CLASSNEXT            (TOOLHELP.21)
 0000:0000  Imp  GLOBALENTRYHANDLE    (TOOLHELP.5)
 0000:0000  Imp  GLOBALNEXT           (TOOLHELP.3)
 0000:0000  Imp  CHECKMENUITEM        (USER.154)
 0000:0000  Imp  GETMENUSTATE         (USER.250)
 0000:0000  Imp  OUTPUTDEBUGSTRING    (KERNEL.115)
 0000:0000  Imp  _wsprintf            (USER.420)
 0000:0000  Imp  SETCURSOR            (USER.69)
 0000:0000  Imp  RELEASEDC            (USER.68)
 0000:0000  Imp  TRANSLATEMESSAGE     (USER.113)
 0000:0000  Imp  POSTQUITMESSAGE      (USER.6)
 0000:0000  Imp  INITTASK             (KERNEL.91)
 0000:0000  Imp  MESSAGEBOX           (USER.1)
 0000:0000  Imp  CLASSFIRST           (TOOLHELP.20)
 0000:0000  Imp  INTERRUPTREGISTER    (TOOLHELP.27)
 0000:0000  Imp  STACKTRACENEXT       (TOOLHELP.19)
 0000:0000  Imp  NOTIFYUNREGISTER     (TOOLHELP.26)
 0000:0000  Imp  LOCALNEXT            (TOOLHELP.9)
 0000:0000  Imp  NOTIFYREGISTER       (TOOLHELP.25)
 0000:0000  Imp  __AHINCR             (KERNEL.114)
 0000:0000  Imp  FATALEXIT            (KERNEL.1)
 0000:0000  Imp  MOVEWINDOW           (USER.56)
 0000:0000  Imp  ENDPAINT             (USER.40)
 0000:0000  Imp  UPDATEWINDOW         (USER.124)
 0000:0000  Imp  GETSYSTEMMETRICS     (USER.179)
 0000:0000  Imp  INTERRUPTUNREGISTER  (TOOLHELP.28)
 0000:0000  Imp  GETDC                (USER.66)
 0000:0000  Imp  SETSCROLLRANGE       (USER.64)
 0000:0000  Imp  GETSTOCKOBJECT       (GDI.87)
 0000:0000  Imp  SETWINDOWWORD        (USER.134)
 0000:0000  Imp  GLOBALFREE           (KERNEL.17)
 0000:0000  Imp  MODULENEXT           (TOOLHELP.11)
 0000:0000  Imp  TASKFIRST            (TOOLHELP.14)
 0000:0000  Imp  GLOBALENTRYMODULE    (TOOLHELP.6)
 0000:0000  Imp  MAKEPROCINSTANCE     (KERNEL.51)
 0000:0000  Imp  LOCALREALLOC         (KERNEL.6)
 0000:0000  Imp  GDIHEAPINFO          (TOOLHELP.23)
 0000:0000  Imp  SCROLLWINDOW         (USER.61)
 0000:0000  Imp  FREEPROCINSTANCE     (KERNEL.52)
 0000:0000  Imp  GETMODULEHANDLE      (KERNEL.47)
 0000:0000  Imp  BEGINPAINT           (USER.39)
 0000:0000  Imp  GLOBALREALLOC        (KERNEL.16)
 0000:0000  Imp  DIALOGBOX            (USER.87)
 0000:0000  Imp  LOCALFREE            (KERNEL.7)
 0000:0000  Imp  APPENDMENU           (USER.411)
 0000:0000  Imp  LOCALINFO            (TOOLHELP.7)
 0000:0000  Imp  MODULEFINDHANDLE     (TOOLHELP.13)
 0000:0000  Imp  TERMINATEAPP         (TOOLHELP.29)
 0000:0000  Imp  LOADICON             (USER.174)
 0000:0000  Imp  LOCKSEGMENT          (KERNEL.23)
 0000:0000  Imp  REGISTERCLASS        (USER.57)
 0000:0000  Imp  LOADCURSOR           (USER.173)
 0000:0000  Imp  SELECTOBJECT         (GDI.45)
 0000:0000  Imp  INITAPP              (USER.5)
 0000:0000  Imp  USERHEAPINFO         (TOOLHELP.22)
 0000:0000  Imp  GETCLIENTRECT        (USER.33)
 0000:0000  Imp  GETSYSTEMMENU        (USER.156)
 0000:0000  Imp  DELETEOBJECT         (GDI.69)
 0000:0000  Imp  LOCALALLOC           (KERNEL.5)
 0000:0000  Imp  TASKFINDHANDLE       (TOOLHELP.16)
 0000:0000  Imp  SHOWCURSOR           (USER.71)
 0000:0000  Imp  INVALIDATERECT       (USER.125)
 0000:0000  Imp  WAITEVENT            (KERNEL.30)
 0000:0000  Imp  SENDMESSAGE          (USER.111)
 0000:0006  Abs  PLOCALHEAP
 0000:0008  Abs  pAtomTable
 0000:000A  Abs  pStackTop
 0000:000C  Abs  pStackMin
 0000:000E  Abs  pStackBot
 0000:9876  Abs  __acrtused2
 0000:9876  Abs  __acrtmsg
 0000:9876  Abs  __acrtused
 0000:9876  Abs  __fptaskdata
 0000:D6D6  Abs  __aDBdoswp
 0001:0010       WINMAIN
 0001:0226       WndProc
 0001:0868       MEMWNDPROC
 0001:0EC4       DUMPMEM
 0001:10B0       _WalkGlobalHeap
 0001:1328       _WalkFreeList
 0001:1530       _WalkLRUList
 0001:1738       _WalkLocalHeap
 0001:1914       _WalkModuleList
 0001:1A16       _WalkTaskList
 0001:1B1A       _WalkClassList
 0001:1C1B       _DoStackTrace
 0001:1D80       _DoUserInfo
 0001:1EA5       _DoGDIInfo
 0001:1FCA       _DoMemManInfo
 0001:21E8       _DoGlobalEntryModuleTest
 0001:225E       _ReadMemoryTest
 0001:230F       _TimerCountTest
 0001:238C       MYNOTIFYHANDLER
 0001:2411       _MyCFaultHandler
 0001:24CB       FAULTDIALOGPROC
 0001:25F4       FAULT
 0001:2670       MYFAULTHANDLER
 0001:26A1       __astart
 0001:270E       _strcpy
 0001:2740       _strlen
 0001:275C       _sprintf
 0001:27B2       _sscanf
 0001:27EC       __cinit
 0001:2899       _exit
 0001:28A0       __exit
 0001:28A8       __cexit
 0001:28B2       __c_exit
 0001:2902       __ctermsub
 0001:2952       __setargv
 0001:2AE0       __setenvp
 0001:2B5E       __flsbuf
 0001:2C3E       __input
 0001:341A       __output
 0001:38F0       __fptrap
 0001:38F6       __aNchkstk
 0001:38F6       __chkstk
 0001:3916       __aFchkstk
 0001:394A       __cintDIV
 0001:394F       __amsg_exit
 0001:396C       __NMSG_TEXT
 0001:3997       __NMSG_WRITE
 0001:39BE       __myalloc
 0001:39EA       __filbuf
 0001:3A7E       __getbuf
 0001:3AC0       _ungetc
 0001:3B20       _lseek
 0001:3B9A       _write
 0001:3CD8       _memset
 0001:3D06       __aNFalmul
 0001:3D06       __aNFaulmul
 0001:3D28       __aNFalshl
 0001:3D46       __dosret0
 0001:3D4E       __dosreturn
 0001:3D5B       __dosretax
 0001:3D68       __maperror
 0001:3D9C       _read
 0001:3E8E       _stackavail
 0001:3EA0       _malloc
 0001:3EA4       __nmalloc
 0001:3EDE       __nfree
 0001:3EEE       __fmalloc
 0001:3F18       __ffree
 0001:3F28       __nrealloc
 0001:3F78       __frealloc
 0001:3FB8       __aNulmul
 0001:3FB8       __aNlmul
 0001:3FEA       __aNlshl
 0001:3FF6       _fflush
 0001:4068       _flushall
 0002:0004       rsrvptrs
 0002:0234       _wListStatus
 0002:0236       _szAppName
 0002:023E       _szMemName
 0002:024A       _szBlockTypes
 0002:0260       _bHasData
 0002:026C       _szLocalFlags
 0002:0276       _szGDI
 0002:028E       _szUser
 0002:02C2       _szNotify
 0002:0930       STKHQQ
 0002:093C       __acfinfo
 0002:094A       __aintdiv
 0002:094E       __fac
 0002:0958       _errno
 0002:095A       __umaskval
 0002:095C       __pspadr
 0002:095E       __psp
 0002:0960       __osversion
 0002:0960       __dosvermajor
 0002:0960       __osmajor
 0002:0961       __dosverminor
 0002:0961       __osminor
 0002:0962       __osmode
 0002:0963       __doserrno
 0002:0963       __oserr
 0002:0965       __nfile
 0002:0967       __osfile
 0002:097B       ___argc
 0002:097D       ___argv
 0002:097F       _environ
 0002:0981       __pgmptr
 0002:0986       __child
 0002:0988       __ovlflag
 0002:0989       __intno
 0002:098A       __ovlvec
 0002:098E       __adbgmsg
 0002:09FC       __aaltstkovr
 0002:09FE       __cfltcvt_tab
 0002:0A0A       __sigintseg
 0002:0A0C       __sigintoff
 0002:0A0E       __asizeC
 0002:0A0F       __asizeD
 0002:0A10       __ctype_
 0002:0A10       __ctype
 0002:0B26       __cflush
 0002:0B28       __amblksiz
 0002:0B2A       __lastiob
 0002:0B2E       __fpinit
 0002:0B3C       ___aDBswpflg
 0002:0B3E       ___aDBswpchk
 0002:0B40       __aDBrterr
 0002:0B42       ___aDBexit
 0002:0B48       ___qczrinit
 0002:0B52       __caption
 0002:0C20       _edata
 0002:0C40       _hInst
 0002:0C42       __iob2
 0002:0CE2       _wsProgramTask
 0002:0CE4       _wsFault
 0002:0CE6       _wNotifyOut
 0002:0CE8       _szText
 0002:0D38       _hwndListStatic
 0002:0D3A       __iob
 0002:0DDA       _wNotifyIn
 0002:0DDC       _hwndMain
 0002:0DDE       _wsFaultTask
 0002:0DE0       _wFilterState
 0002:0DE2       _wsIP
 0002:0DE4       _wsCS
 0002:0DE6       _hwndList
 0002:0DE8       _hwndListLocal
 0002:0DEA       _xChar
 0002:0DEC       _xScreen
 0002:0DEE       _yChar
 0002:0DF0       _yScreen
 0002:0DF2       _wNotifyState
 0002:0DF4       _end

Program entry point at 0001:26A1
